:101800003BC06FC054C053C052C051C050C04FC045
:101810004EC04DC04CC04BC04AC049C048C047C074
:1018200046C045C044C0040309041C037700770088
:1018300077002E00660069007300630068006C008A
:101840002E00640065000E03550053004200610045
:101850007300700012011001FF000008C016DC05C3
:101860000201010200010902120001010080320997
:10187000040000000000000011241FBECFE5D4E0EA
:10188000DEBFCDBF10E0A0E6B0E0EEE2FFE102C0B7
:1018900005900D92A636B107D9F710E0A6E6B0E0A4
:1018A00001C01D92AC39B107E1F754D13EC3A8CFB6
:1018B000A82FB92F80E090E041E050EA609530E039
:1018C00009C02D9182279795879510F08427952739
:1018D000305EC8F36F5FA8F30895EADF8D939D93A0
:1018E0000895CF93CFB7CF93C395849BE9F7849B9B
:1018F00009C0849B07C0849B05C0849B03C0849B54
:1019000001C0A1C0DF93C0917F00DD27CA57DF4F20
:10191000849B02C0DF91EBCF2F930F931F9300B3F3
:101920002FEF04FB20F94F933F9310B34FEF0127A4
:1019300004FB21F93BE031C04E7F012F10B3216041
:1019400028C0102F4D7F2260000000B329C04B7FBC
:101950002460012F000010B32BC010B3477F286014
:101960002AC04F7E00B320612CC04F7D10B320628F
:101970002FC04F7B00B3206432C0422700B349938D
:101980004FEF0000102714FB20F910B31471C9F1B8
:10199000297F91F2012704FB21F900B3237F89F20B
:1019A000315058F1102714FB22F910B3277E79F239
:1019B000012704FB23F92F7C81F200B3102714FBCD
:1019C00024F92F7971F200C010B3012704FB25F927
:1019D0002F7359F200C000B3102714FB26F92230F0
:1019E00040F200C010B3012704FB27F9243028F689
:1019F0004F77206810B30000F9CF10E41ABF00271A
:101A000017C03B503195C31BD04010E41ABF08816A
:101A1000033CE9F00B34D9F020917D001981110FBE
:101A20001213EDCF093641F10D3211F0013E39F7B5
:101A3000009384003F914F911F910F912F91DF915F
:101A4000CAB7C6FD51CFCF91CFBFCF911895209186
:101A50008400222379F310918200112311F5343090
:101A600012F13093820020937E0010917F003BE0C2
:101A7000311B30937F0017C00091820001308CF43D
:101A80000AE53091600034FD10C000936000C2E7A9
:101A9000D0E00FC02795A8F45150A9F4220F000000
:101AA000F9CF4AE503C042ED01C0432FC4E1D0E0C5
:101AB00032E011B31461949A11BB02B320E414E133
:101AC0005F93012756E002BB279520F4515021F483
:101AD000220FF9CF012756E000003B5A02BBD0F29B
:101AE000279528F4515029F4220F0000F9CF01273F
:101AF00056E0279502BB20F4515021F4220FF9CF74
:101B0000012756E02991332302BB21F60B7E109169
:101B10008300110FC651D04002BB11F010937D001D
:101B200010E41ABF006111B31B7E402F4B7E5F9102
:101B300000C000C002BB11BB42BB7CCF12BAF894FC
:101B40001BBE15BE81E08BBF1BBEE0917000F09103
:101B50007100099588E10FB6F89481BD11BC0FBEE4
:101B6000979A04B601FECBC114BE81E08BBF82E020
:101B70008BBF8799C4C185B7826085BF8BB78064EE
:101B80008BBF8C9A20E005C0A89588EB9BE001975D
:101B9000F1F72150C9F78C987894FF2400E09091D8
:101BA0008200935097FD2EC180917F00CCE0D0E061
:101BB000C81BD109CA57DF4F80917E008D3209F0D2
:101BC000C4C0983009F01CC183EC809372008AE590
:101BD0008093600010926A003881832F807629817B
:101BE000882309F443C086E690E0909381008093B7
:101BF00080002330C9F49B818C812A81203339F401
:101C00008370E82FF0E0EE59FF4F808109C0203A41
:101C100011F476D105C0203C11F46D8179D180E0BA
:101C20008093690094E087C0253011F491E083C06F
:101C3000822F8450863098F48A819B8190936D0026
:101C400080936C00293081F09E8190936E008D818D
:101C5000827080936F0037FD69C02FEF68C022301B
:101C600019F481E080936B0090E065C08A81109246
:101C70007B00222331F410927C002BE730E092E0CD
:101C800050C0253019F48093830048C02630B1F548
:101C90008B81813019F484E598E104C0823041F4ED
:101CA00086E698E1909381008093800092E122C0C3
:101CB0008330F9F48A81882341F486E298E1909395
:101CC00081008093800094E015C0813041F48AE265
:101CD00098E190938100809380009CE10BC082305A
:101CE00041F486E498E190938100809380009EE027
:101CF00001C090E080E480936A001DC0283019F490
:101D000025E830E009C0293019F48093850006C029
:101D10002A3021F42BE730E091E003C02BE730E0DC
:101D200090E0309381002093800005C0292F80E847
:101D300080936A0007C08F81882319F42E812917A8
:101D400008F0292F209361005BC080916A0087FF13
:101D500057C080916E00592F891708F4582F851BA2
:101D600080936E0060E0882309F461E070916F0059
:101D7000E0916C00F0916D0040E037C0CF018F73AF
:101D80009070892B49F4F89483E080935700E8958C
:101D9000789407B600FCFDCF4E5FF8948991999135
:101DA00021E00C0120935700E895112478949F01BD
:101DB0002E5F3F4FC9018F739070892B31F06623DE
:101DC00099F0451788F0772379F0F89485E08093AF
:101DD0005700E895789407B600FCFDCFF89481E1B0
:101DE00080935700E8957894F901451708F4C6CF19
:101DF000F0936D00E0936C00662311F01092610087
:101E0000109282008091600084FF65C08091610023
:101E10008F3F09F460C0182F893008F018E0811B4B
:101E2000809361008091720098E889278093720006
:101E3000112309F43EC080916A0087FF1EC0809183
:101E40006E00811708F4182F811B80936E00E091BB
:101E50006C00F0916D00A3E7B0E003C084918D9316
:101E60003196812F90E08D589F4FA817B907B1F791
:101E7000F0936D00E0936C001AC0E0918000F09147
:101E8000810086FF09C0912FA3E7B0E084918D9374
:101E900031969150D9F707C0912FA3E7B0E0819117
:101EA0008D939150E1F7F0938100E0938000193019
:101EB00060F483E790E0612F10DD612F6C5F6C3080
:101EC00041F08FEF8093610004C08FEF8093610039
:101ED0006EE16093600094E180B3847131F49150BD
:101EE000D9F71092830010927D0080916B008823B7
:101EF00021F0FA9411F4015011F0879B50CE1EDEB0
:101F0000E199FECF9FBB8EBBE09A99278DB30895D0
:101F1000262FE199FECF9FBB8EBB2DBB0FB6F89449
:0E1F2000E29AE19A0FBE01960895F894FFCF61
:061F2E005AFF1E9307009C
:0400000300001800E1
:00000001FF
